:10000000000000308A002029FF00030E8312031332
:10001000A1000A08A0008A010408A2007708A30032
:100020007808A4007908A5007A08A6007B08A70034
:10003000831383120B1E1E288B184D288B1E22281B
:100040000B1950288C308400801C28288C185628C6
:100050008C308400001C2E280C1853288C3084000F
:10006000801E34288C1A5C288C308400001E3A28AC
:100070000C1A5928220884002308F7002408F800E5
:100080002508F9002608FA002708FB0020088A0046
:10009000210E8300FF0E7F0E09000A128A11A2288A
:1000A0000A128A11E1280A128A1170280A128A118A
:1000B000B2280A128A117F280A128A1166280A10A9
:1000C0008A100A11820753344C343034A808031DB7
:1000D0006C281A08A8006D2807128A110A123A28FB
:1000E000831698128312871287151816D030A9002C
:1000F0008C30840000100C108A110A123A282A1D34
:100100008A28FC308F0069308E008C308400001407
:100110002A119F28F0302902031C912807122A1562
:100120009F28831729088400000899002908840063
:100130000D300002031D9E282A159F28A90A8A1146
:100140000A123A28910188308316920008308312EF
:10015000AB0006120B128C30840080148B108A11B5
:100160000A123A28AB08031DCA288C30840080107C
:100170000B1683172C0884000D3000020319C628C3
:100180002C0884000A300002031DC8282A14061611
:10019000AC0ADD28C1010618C10A00000618C10A10
:1001A00000000618C10A00008317C118D9280310DF
:1001B000DA2803142C088400800C8C108A110A128F
:1001C0003A287C3081000030AA180130F700013055
:1001D0007702031DF3288610061586128B16AA10C7
:1001E0000830AB001429AB08031D04290611AA141A
:1001F00083172C0884000D300002031D03298B1285
:100200009030AC0086161429AB0B082986141429EB
:1002100083172C088400003084070310800C031817
:1002200013298610142986140B118A110A123A28F0
:100230003F1F1C290930BF073F080F39F800003461
:1002400084011F3083059F308400073080008501C2
:10025000303086001D308700FF306500C9306600F1
:10026000823067000830F700F71D3E290730810112
:10027000813084000008C0390F388000640081306C
:1002800084000008C03977048000053090000030F9
:10029000F800780804389200FF3083169200173077
:1002A000990006309800903083129800B6143611E9
:1002B0002A11A8011030B000FF30B100FF30B200A9
:1002C000D030A9008C30840080168C308400001659
:1002D000C0308B04A8080319162A2808B300A80107
:1002E000B61C8C292330330203197A2921303302BA
:1002F000031D8B2907119030AD00AE01B6103611E9
:1003000023303302031D88290330AF0036148B29B4
:100310000130AF003610162A31083002031D932930
:1003200007123615072A0D30330203199B290A30AC
:100330003302031DCC2904302F072E020318A229F3
:100340003615C929361CB7293408BF00182178088A
:10035000BE00BE0EF030BE053508BF0018213E08B5
:100360007804AD07AD080319B729361507123619F9
:10037000C9298317300884000D3080003008B2008E
:100380006F303002031DC7291030B000C829B00AF1
:100390000716B6140715072A02302E020318D829AB
:1003A000361CD82934302E07840033088000E92910
:1003B0002E082F020319DE290318E92903302F071D
:1003C0002E020318E9292F082E025F203302031D95
:1003D0003615361CF12907302E02031CF12933088B
:1003E000AD073619062A04302F072E02031C062AF1
:1003F000831730088400330880003008B00AF70003
:1004000070307702031C062A1030B000AE0A361D89
:10041000162A6F303202031D102A1030B000132A42
:1004200001303207B000B614071536113108320218
:100430000319632B310A031D202A1030B100212A31
:10044000B10A8317310884000008F70051307702A1
:100450000319332A533077020319A72A4E30770243
:100460000319522B532BD03029020319392A0712B2
:10047000A62A83172908A90A840054308000290875
:10048000A90A8400683080002908A90A8400653020
:1004900080002908A90A8400723080002908A90A6E
:1004A00084006D3080002908A90A84006F30800024
:1004B0002908A90A8400733080002908A90A840049
:1004C000743080002908A90A84006130800029085E
:1004D000A90A8400743080002908A90A8400203009
:1004E00080002908A90A8400513080002908A90A3F
:1004F0008400753080002908A90A840065308000D6
:100500002908A90A8400723080002908A90A8400F9
:10051000793080002908A90A840020308000290849
:10052000A90A84004F3080002908A90A84004B30B2
:1005300080002908A90A84000D308000D030A9006D
:10054000871118128716831698168312552B831756
:10055000320831020319B92A310884000D30000233
:100560000319B92AB10A70303102031CB92A1030BC
:10057000B100310884000008B700320831020319C5
:10058000CE2A310884000D3000020319CE2AB10AA8
:1005900070303102031CCE2A1030B10031088400C3
:1005A0000008B800320831020319E32A3108840038
:1005B0000D3000020319E32AB10A70303102031C26
:1005C000E32A1030B100310884000008B900320875
:1005D00031020319F82A310884000D300002031992
:1005E000F82AB10A70303102031CF82A1030B10029
:1005F000BD01310884000D3000020319292B03309E
:100600003D020318292B320831020319142B31083B
:1006100084000D3000020319142BB10A703031022E
:10062000031C142B1030B100310884000008B30003
:100630000B138B138B1B192B83133D08BD0AF7007B
:100640003A3077078400330880008317C0308B046A
:10065000F92A3708F700413077020319482B433055
:1006600077020319492B4630770203194A2B483089
:10067000770203194B2B4C30770203194C2B4D306A
:10068000770203194D2B5330770203194E2B4F2B52
:10069000512B512B512B512B512B512B512B0712DD
:1006A000512B552B552B0712552B310884000D303B
:1006B00000020319632BB10A70303102031C622B54
:0C06C0001030B100552B6A296300630064
:02400E00333548
:084000000000000006000400AE
:00000001FF
